:020000040100F9
:10000000FD62938202400100FD12E39E02FE374131
:10001000000213010100B701000293810100B7152E
:100020000001938505F137160001130606F4B706A3
:1000300000029386060039A083A2050023A0560083
:1000400091059106E3EAC5FEB7150001938505F415
:1000500037160001130606F4B7060002938606263B
:1000600039A083A2050023A0560091059106E3EA7A
:10007000C5FEB70500029385050337060002130687
:10008000062621A023A005009105E3EDC5FEB700DB
:100090000001E780C00AB7000001E780C00AB7008E
:1000A0000001E780007273005010F5BF82800000ED
:1000B0000000000000000000000000000000000040
:1000C0006F004000197106C20AC40EC612C816CAD3
:1000D0001ACC1ECE22D026D22AD42ED632D836DA48
:1000E0003ADC3EDEC2C0C6C2CAC4CEC6D2C8D6CA78
:1000F000DACCDECEE2D0E6D2EAD4EED6F2D8F6DA28
:10010000FADCFEDE970000009380E00482909240CB
:100110002241B2414242D2426243F24302549254DB
:100120002255B2554256D2566257F2570648964863
:100130002649B649464AD64A664BF64B065C965C5B
:10014000265DB65D465ED65E665FF65F096173004A
:10015000203001A03D432A876373C3029377F700E1
:10016000BDEFADE5937606FF3D8ABA960CC34CC34E
:100170000CC74CC74107E36BD7FE11E28280B30680
:10018000C3408A069702000096966780A600230760
:10019000B700A306B7002306B700A305B7002305E1
:1001A000B700A304B7002304B700A303B7002303D9
:1001B000B700A302B7002302B700A301B7002301D1
:1001C000B700A300B7002300B700828093F5F50FB6
:1001D00093968500D58D93960501D58D61B793963D
:1001E00027009702000096968682E78086FA96801E
:1001F000C1171D8F3E96E374C3F8A5B7B707050076
:100200000947D8CFB7170500938707C0984385667D
:1002100093860640558F98C3B71708009387074009
:1002200023A0070023A2070023A407001307A008A8
:10023000D8C77D57D8CF354798C3D84F9356570165
:100240008D8AE5DE8280B71708009387074023A0D8
:10025000070023A2070023A4070023A607007D5759
:10026000D8CF23A40702B7170500938707C0984388
:10027000F1769386F63F758F98C3B7070500D84F80
:1002800023AE07008280B71708009387074088D7FE
:10029000D84F137707046DDF828037070002B71548
:1002A000080037460F0023200704814781469385C5
:1002B000054013061624C84D137505020DC991CECD
:1002C0002320F70437470F00130707246397E7003D
:1002D000B707000205472383E700B7170800938795
:1002E0000740C8534205418182808546E9B78507AA
:1002F000E39DC7FEFDD2B7470F0093870724232055
:10030000F704F9B74111B707000222C413870700A9
:1003100006C6834667000547138407006390E6021C
:100320001305000F8D37B717080093870740D84F84
:10033000218B09C7D84F13678700D8CF2303040048
:10034000B240224441018280411106C622C426C225
:10035000AA84EF009013E1689388086A01488147F6
:10036000014781460146B70520C726853794980086
:10037000EF000077130414687D1419E40D45B240B2
:10038000224492444101828085452685EF00501128
:1003900005897DF10145E5B7411122C4370400020A
:1003A000930704008C43B70700804AC0BE95B70787
:1003B000000223ACB70206C626C293974501130478
:1003C00004003709000289E713058900EF00701A5D
:1003D0000C40B70400029386440413060010130572
:1003E0008900EF0050141C40370700028356470372
:1003F000938707101CC013060010B68763F4C6006D
:1004000093070010138444041305F400938707F046
:100410001306100F814513040410231AF7021D3B25
:10042000A285138544043D46EF00F0182320040004
:1004300023220400232404002316040023070400BD
:10044000B240224492440249410182805D71130608
:1004500080028145280886C6F539BD47230CF10086
:100460008947230EF1003ED2E177938707082C08D5
:100470000A85231AF1021923B640616182805D71F9
:10048000A2C4370400021305840086C6A6C2652BE9
:1004900013058400E525894513058400EF0050000D
:1004A0009377250085E3AA84854513058400EF0032
:1004B000207F13E62400AA851376F60F1305840027
:1004C000EF007001E1689388086A0148814701479D
:1004D00081460146B7052038130584001125E168DF
:1004E00038009388086A1308000285468147014650
:1004F000B70599EB1305840023040100D523B71534
:10050000000151469385C5EF6800EF00D00A9304BF
:1005100084009C406C0051463ED085473ED2681016
:10052000C1673ED4EF003009B70607009C42370789
:10053000F1FF7D17F98F08109CC2812BB64026442D
:10054000964461618280411106C6F5390D3FB707B7
:10055000008073905730B70000808290B240410114
:100560008280411106C622C426C24AC08347350094
:1005700005476383E70811472A846389E7008DCF25
:10058000B24022449244024941018280B7070002EE
:1005900083D7470391C30935834744000347540079
:1005A000E2074207BA9737070002232EF702370700
:1005B00000022320F700E9B73709000283544903FA
:1005C0000346050093054500370500021305450461
:1005D0002695EF00407E83470400BE94C204C1808C
:1005E000231A99029307F00FE3FC97F82244B240D4
:1005F0009244024941014DB33D457131B7070002B4
:1006000083D7470391C3493B2244B24092440249F5
:10061000410115BF3707000293070700B705000225
:1006200003DE470083A705043716080037450F008F
:1006300037480F00B708000201438146130707003F
:10064000130606401305152413080824938848153B
:1006500063EEC6016304030023A0F504834767002B
:10066000A9E73705000213054515E5BD81470323BA
:10067000C60113730302631F03008507E399A7FEF6
:10068000B7470F009387072423A0F504854723036A
:10069000F7008280E38607FF832E46023383D8006B
:1006A00085062300D301054365B78280011122CC62
:1006B0003704000226CA4AC84EC652C406CE1304E6
:1006C0000400930400061309E00FB7090002130A9F
:1006D0000003E136834764001375F50FA303A400FC
:1006E00099C30D31FDB7630F950063042503E31231
:1006F00045FF3D45493E553605052312A4003D45BD
:100700005936C1BF3D454136313783476400F1FB5F
:10071000FDB7138589000D397DD11305000FCDB7C5
:10072000011106CE22CC1D333704000213058400CC
:10073000192E130584009921E1689388086A0148FD
:100740008147780085460146B705D9EB130584003B
:10075000230601007126E168814701478146014671
:10076000B70538FF9388086A0148130584008D2E69
:10077000713437070002B715080037460F002320F1
:100780000704814781469385054013061624C84D0A
:100790001375050211CD85CA2320F70437470F00D2
:1007A000130707246391E702793B01A08546C5B78B
:1007B0008507E39DC7FE81CAB7470F0093870724CB
:1007C0002320F704D5B7DD350547AA876305E50281
:1007D00009476300E506054591EBB7060600DC4ACC
:1007E0007D771307F73FF98FDCCA014582807D17BB
:1007F00019EB0D4582809306004037A707001307C9
:100800000712B7050500905D7D8E75D2370606008C
:100810005C4A7D771307F73FF98FD58F41115CCA8A
:1008200002C613073006B2476359F700014541017C
:100830008280856693860680C9B7B24785073EC623
:10084000DDB791476307F50263EAA7008547630AAE
:10085000F50489476309F50405458280A147E31D36
:10086000F5FE0947094501A8FD1781EFC8D20D45DE
:10087000828005470D45B7A7070093870712B70683
:100880000500905E798E6DD28A05C98D4111CCD25A
:1008900002C613073006B247635AF700014541010B
:1008A00082801147C9BF21470145F1B7B24785078B
:1008B0003EC6D5B70547AA876305E5020947630227
:1008C000E506054591EBB70606009C4A7D771307C0
:1008D000F73FF98F9CCA014582807D1719EB0D45C2
:1008E00082809306004037A7070013070712B70559
:1008F0000500905D7D8E75D2370706001C4B7D7616
:100900001306F63FF18FD58F1CCB85471CCF4111C5
:1009100002C613073006B2476359F700014541018B
:1009200082808566938606807DBFB24785073EC676
:10093000DDB711C98547630DF50205458280FD17B6
:1009400091EB0D4582800946B7A7070093870712F0
:10095000B7060500985E718F7DD34111C8D602C6D7
:1009600013073006B2476357F70001454101828003
:100970000546D9BFB24785073EC6EDB7011126CA65
:10098000B7040600DC4806CE22CC4AC84EC652C484
:1009900056C2F19BDCC89C482A89C845F19B9CC87B
:1009A00083C7C5012E848A07DCC883C7D5018A079F
:1009B0009CC8193D0C44AA8A03454400593518487F
:1009C000B70705002A8A98C358480850D8C3184C5E
:1009D00098C7CD35AA894850A93F834704002A8784
:1009E00093F6170089E6D44893E62600D4C893F618
:1009F000270099E637060600544A93E6160054CAC3
:100A000093F6470099E637060600144A93E6260057
:100A100014CAA18B99E7B70606009C4A93E7170012
:100A20009CCAF24062442320590123224901232415
:100A300039012326E900D244B249224A924A4A8522
:100A4000424905618280011106CE22CC02C402C651
:100A50002147B707050037550800D8C705448D471B
:100A60008A85130505803EC022C2292A3755080011
:100A70009307C0038A851305058022C222C43EC0A5
:100A80001122F240624405618280411122C406C6EF
:100A90002A84553F18405C4F93E707015CCF1C4404
:100AA0001CCB5C4085CB1C43B7061000D58F1CC304
:100AB000144C5C48B240D606CE07D58F834604015D
:100AC000C206D58F8346C4012244E206D58F1CCFCF
:100AD000410182801C43B706F0FFFD16F58FC1BFB0
:100AE000032305002A8E0325C30113650502232E67
:100AF000A3002324C3001396260149824D8E23268A
:100B000003012322C300139605016354060299C210
:100B10000545B1CB01476346D700639C08020D45EC
:100B200082803386E700034606000507230AC300D8
:100B3000DDB799C2054505CB8147E3D0D7FE032633
:100B40000E00034546013306F70085072300A60083
:100B5000EDB783270E00FD18DC4F93F70702D5DFB2
:100B600011656D8D11E18280B707070083C74701CA
:100B700013F585001D8D3335A00082801C4141474F
:100B8000D8CF8280B7470800938707402A8863043C
:100B9000F508B7570800938707806304F50A3747BD
:100BA0000800630DE50A05458280331E1F01337678
:100BB000DE0129C683A345008843139318003396AA
:100BC0006F001346F6FF13F43300718D3314640085
:100BD000418D88C3638B5302638C0302084303AEC9
:100BE000C500718D331E6E003365C50108C3884290
:100BF000698E884533156500498E90C2850833D5C6
:100C00001E0145F53244410182802326C801F9B70F
:100C10002324C801E1B7B716050037170500B71739
:100C20000500938646C1130707C19387C7C083AEEB
:100C300005008148054F8D4F914233D51E0105EDCA
:100C40008280B716050037170500B7170500938691
:100C500006C21307C7C1938787C1D1BFB716050066
:100C600037170500B7170500938686C0130747C0DE
:100C7000938707C06DBF331E1F013376DE0119E273
:100C8000850865BF411122C635B7E1689388086AB7
:100C900001488147014781460146B705200689B5CD
:100CA000011106CEA307010089476393F502B7053A
:100CB0002035E1681307F1009388086A01488147ED
:100CC00085460146313DF2400345F10005618280D1
:100CD000B7052005F9BF011106CE22CC26CA23068E
:100CE000B100AA84A306C1004D37E1689388086A61
:100CF00001487C00014789460146B78520012685C9
:100D00000964F93B130414717D1419E40D45F24094
:100D10006244D24405618280854526855137058924
:100D200065F50145EDB7011106CE22CC26CA2E8409
:100D30004AC8AA84328936C6893FB247E16822860A
:100D40009388086A01480147CA86B78580022685CC
:100D5000616479331304146A7D1411C485452685B2
:100D60008137058975F9F2406244D24442490561F0
:100D70008280011106CE22CC26CA2EC6AA84313723
:100D80003246E1689388086A0148814701478146F5
:100D9000B705802026856164A1331304146A7D148D
:100DA00011C485452685ED3D058975F9F2406244FB
:100DB000D24405618280B3C7A5008D8BB308C500FE
:100DC000B1E78D4763F4C704937735002A87B9EB01
:100DD00013F6C8FFB306E6409307000263C8D706C0
:100DE000AE86BA876371C70203A806009107910611
:100DF00023AE07FFE3EAC7FE9307F6FF998FF19B47
:100E000091073E97BE956366170182802A87637EAD
:100E1000150383C7050005078505A30FF7FEE39AB1
:100E2000E8FE828083C60500050793773700A30F8D
:100E3000D7FE8505D1DF83C6050005079377370008
:100E4000A30FD7FE8505F9FF61B78280411122C645
:100E50001304000283A3050083A2450083AF85002D
:100E600003AFC50083AE050103AE450103A38501B1
:100E700003A8C501945113074702B307E640232E88
:100E800077FC232057FE2322F7FF2324E7FF2326A6
:100E9000D7FF2328C7FF232A67FE232C07FF232E13
:100EA000D7FE93854502E347F4FAAE86BA876371AD
:100EB000C70203A806009107910623AE07FFE3EAE5
:100EC000C7FE9307F6FF998FF19B91073E97BE955A
:100ED0006365170132444101828083C7050005071D
:100EE0008505A30FF7FEE387E8FE83C70500050726
:100EF0008505A30FF7FEE392E8FEE9BF200000009E
:100F0000010000000300000006000000EB000000EC
:100F10000000008000010000000007000000000049
:100F200000000000000000000000000000000000C1
:100F300000000000000000000000000000000000B1
:0400000501000000F6
:00000001FF
